:020000020000FC
:1000000011C018951895189512C11895189587C0A4
:10001000189507C11895189518951895189518955D
:100020001895189512E00FE51EBF0DBFA89508E1C1
:1000300001BD0EE101BDA895B0E0A0E610E000E42E
:100040001D930A95E9F70FEF0ABB00270BBB03E0EE
:1000500007BB002704BB0FEF05BB04EF01BB08E0A3
:1000600002BB01E006B90FEF07B903E003BF09E1E6
:100070000BBD04E60ABD00270FBD0BE00EBD02E478
:1000800009BF01E009B900E000BD0EE800BD22276C
:100090006CB12BB9579A549A1124442757E0E0E6E3
:1000A000F0E030E08FEFA895789436FD01C0FDCFE9
:1000B0003F7B326073FD30C074FD2BC0213029F0CE
:1000C000223061F0233078F4F0CF662329F52395B0
:1000D000A3B3A095BB272A9BB395E7CF1197A1F7B0
:1000E000B0E0A0E623957C91671711F06C9330681F
:1000F0001196839907C0A03A39F7B03029F73160DB
:100100002227D3CFA83701F7B030F1F6316022278C
:10011000CCCF5C9821E0C9CF22275B98C6CF9FB691
:10012000440F09F04FC01BBA839925C0539558302E
:10013000E8F4949A01910093B00001910093B1000A
:1001400001910093B20001910093B30001910093DB
:10015000B40001910093B50001910093B6000191A4
:100160000093B70042E0959894982CC0959A552733
:10017000E0E6F0E0DECF550F583000F5052F029590
:1001800012B31F78102B12BB01910093B0000281B3
:100190000093B10005810093B20000850093B30085
:1001A00003850093B40006850093B5000189009390
:1001B000B60004890093B70042E004C051E0E0E6D5
:1001C000F0E0DCCF142F109512BF11270091B00082
:1001D000042309F011600091B100042309F01260BA
:1001E0000091B200042309F014600091B3000423CD
:1001F00009F018600091B400042309F01061009127
:10020000B500042309F010620091B600042309F040
:1002100010640091B700042309F010681BBB9FBE57
:1002200018959FB67BB16CB130649FBE18959FB690
:10023000A89537FD11C0389A80FD02C0979A01C079
:1002400097988695813031F480E830FF85E831FF5A
:1002500081E83C7F9FBE18953F77389B02C0389855
:08026000EBCF389AE9CFFFCF84
:00000001FF
